:020000040000FA
:06000000ADEF04F0120058
:060008009AEF04F0120063
:060018009AEF04F0120053
:06082A0001008609000038
:080830006A0000000400000052
:080838002A0EF66E080EF76EA1
:10084000000EF86E00010900F550656F0900F550C3
:10085000666F03E1656701D03DD00900F550606F18
:100860000900F550616F0900F550626F0900090039
:10087000F550E96E0900F550EA6E0900090009001B
:10088000F550636F0900F550646F09000900F6CF59
:1008900067F0F7CF68F0F8CF69F060C0F6FF61C08D
:1008A000F7FF62C0F8FF0001635302E1645307E001
:1008B0000900F550EE6E6307F8E26407F9D767C0E8
:1008C000F6FF68C0F7FF69C0F8FF00016507000E7A
:0608D000665BBFD71200B9
:0A08D6001200D9CFE6FFE1CFD9FFF1
:1008E000FD0EDBCF02F0DB06FE0EDBCF03F001E2F4
:1008F000DB060250031001E0F3D7E552E7CFD9FF42
:100900001200870ED56E880ED56EE00EF26E1200C4
:10091000F00E951600016D716D516A256A25020170
:10092000006F6CC000F200C283FF1200EADFF0DF4C
:10093000FED71200DACFE4FFE2CFDAFFE652E40E90
:10094000D66E480ED76E00016A2B6B2B000E6C23FF
:0A095000F294E552E5CFDAFF110042
:06095A0013EE00F023EE95
:1009600000F0F86A019C1CEC04F0C2EC04F096EC78
:0609700004F0FBD71200A9
:0A09760000EE00F00F0EEE6AEA62D8
:04098000FDD712008D
:0209840012005F
:04098600000000006D
:00000001FF
